:020000040000FA
:0400000024280000B0
:08000800FD00030EFE000A08D2
:10001000FF008A0183010B130C1C102840200C10D8
:100020000B1C16288A1516268A110B108C1C1C28EE
:100030008A1580268A118C107F088A000B177E0E85
:100040008300FD0E7D0E09008316031331308500F9
:1000500096308600831603138113831203138501E0
:1000600086018316031307309C009B018312031340
:1000700006178A15042665108A1595268A116028A8
:10008000FF308F008316A40B4E282508A4002308F8
:10009000A20083128E008316A10A5228220883121E
:1000A0008E008316A00AA01959288312851408000F
:0800B0005C2883128510080092
:1000C000831603133030850083120313051483163F
:1000D000031316308600A225A225A2258316031736
:1000E0000030900094009300EF01C8268A159728ED
:1000F000831603139630860083120313C601C701CB
:100100008312DB01C301C401C501EE01F50137080B
:10011000EF003608F0004D14CD1483120317481079
:10012000C810722283160317E501E601E901EA010E
:10013000E503E60383120313F40183120313861508
:100140008230831203178D008312031374278316E2
:100150000317A000A01DAF288316031769164B30A4
:100160005C27542984000008080082078207303485
:100170003034323437340034820742344C3447341C
:1001800050345334303400348207FC347C343C34F3
:100190001C340C3404348434C434E434F434831212
:1001A00003136518D428D6287421CF282A30831643
:1001B00003176F1CDD284630E428691FE1285E30F4
:1001C000E428E91FE428563083120313401AEC2870
:1001D00083160317D500EF2883160317D3005C2777
:1001E000492383120313F50183120313D200013C48
:1001F000031D092983120313C01FFF28092383123B
:100200000313C01C092983160317E91B09298A1542
:10021000422B831203134D1C17295208013C031D66
:10022000172983120313C01E17298A15162A831251
:100230000313CD1C3229CD108B26831203130130FA
:100240009000EF3092000B17831603130C148C14DC
:1002500083120313401B2E297F24202683160313A9
:100260000C10831283120313401D53291F2783127E
:1002700003134108460203193E2953294708420245
:100280000318432953295A305C278316031361301E
:100290008F0083120313861183160313FF3085002A
:1002A000F73086006300CF280030D7005829D70ADE
:1002B0005708503C031C6529A225831203136518B7
:1002C0006229642974215F29572950308E008316D2
:1002D000A200A3008312FF308F000B1783160313B5
:1002E0000C14831203137B2C542783120313313A0B
:1002F000031D7C29EA29EA29313A3F3A031D822964
:10030000662CEA293F3A4D3A031D88296D2CEA29CB
:100310004D3A563A031D8E29642CEA29563A543A2E
:10032000031D9429262CEA29543A503A031D9A2990
:10033000562AEA29503A473A031DA0297B2CEA297C
:10034000473A533A031DA6290D2AEA29533A443A5B
:10035000031DAC29F929EA29443A5A3A031DB32965
:100360008A154228EA295A3A553A031DB929352AED
:10037000EA29553A433A031DBF29212AEA29433A7B
:10038000423A031DC6298A15002FEA29423A573AF4
:10039000031DCC29392CEA29573A583A031DD22992
:1003A000502CEA29583A493A031DD9298A15E528DB
:1003B000EA29493A4A3A031DE0298A150029EA291F
:1003C0004A3A4B3A031DE7298A158D28EA294B3A08
:1003D00008002428ED218625EB2983120313013020
:1003E00090008312F5250B17831603130C14831644
:1003F0000800831203138B30D700FF29D70A570850
:100400008E3C031C0C2A5708831203178D0083129D
:10041000031374275C27FE296F2C8312031380308B
:10042000D700132AD70A5708833C031C202A5708F1
:10043000831203178D008312031374275C27122A7B
:100440006F2C831203138430D700272AD70A57084A
:100450008A3C031C342A5708831203178D00831229
:10046000031374275C27262A6F2C0A305C270D3073
:100470005C2783120313831203132030840083123A
:1004800003130030D500452AD50A55080E3C031C3D
:10049000532A83120313651C4B2A54278312031318
:1004A0008000840A442AF526C8266F2C0A305C276F
:1004B0000D305C2783120313203084000030D500F8
:1004C000622AD50A5508223C031C702A83120313A2
:1004D000651C682A5427831203138000840A612A4A
:1004E0000A276F2C831603134030990083120313DD
:1004F00090309800181218168316031320309800B5
:10050000831203130800952A8312031375088A15B2
:1005100000208A115C2775088A1500208A11F50AC7
:10052000080083228000840A08004030CA006E0858
:1005300045020319B22A831203134508EE00031D76
:10054000A62AC818A62AC8140030C507EF03031D41
:10055000AC2ACD143708EF00F003031DB22A4D1466
:100560003608F000CA0B972ACF0B842A8F30CF00B1
:10057000D10B842A54305C274F30C12A4E305C277F
:1005800044305C2700300800831783120313BF3008
:10059000D9006130DA001D30D5001A24831383128C
:1005A00003138312031383130800831783120313A7
:1005B000401EE42A831203132030D9009F30DA0052
:1005C0001C30D5001A24ED2A831203132030D900E1
:1005D0009F30DA001D30D5001A2483132D3083128A
:1005E0000313401AF72A83160317D500FA2A831635
:1005F0000317D30083138312031308008322F1002F
:100600008322F1078322F1078322F1078322F10776
:10061000080083120313CF01FF30D700D70B112B33
:10062000BE2A97258322243C031D0E2BFE228830F0
:10063000710203191C2B0E2B8322832283120317B2
:10064000BD00832283120317BE0083228312031787
:10065000BF000C240C240C240C24832283120317C7
:10066000C000832283120317C10083228312031761
:10067000C2000800832283160317EC00832283162E
:100680000317ED00EE018A15D2228A118312031797
:10069000080083120313CF0118121816FF30D70079
:1006A000D70B532BBE2A97258322243C031D502BA6
:1006B000FE226630710203195E2B502B83228322A7
:1006C00083160317EC002C3C031D672BD52B3E2310
:1006D000C5003A23C4003A23C3008A110C248317AF
:1006E000BF3084000030D500762BD50A5508063C73
:1006F000031C812B832280002C3C0319D52B840AF8
:10070000752B83120313401A882B912291228C2B74
:100710008322E9008322EA008322912283160317B1
:10072000E910533C031D952BE9148322840A003001
:10073000D5009B2BD50A5508073C031CA12B912201
:100740009A2B83120313401AA82B91229122AC2BCF
:100750008322EB008322EC0083229122831603176D
:100760006911573C031DB52B69150C240C248322F9
:1007700083160317EC00832283160317ED008322F0
:100780000C2483120313401AC72BD630C82BD63043
:1007900084000030D500CD2BD50A5508043C031C3D
:1007A000D32B9122CC2B1124DB2B1124D5228316A1
:1007B0000313B101C22AC4228316031742238316EE
:1007C0000313B100831203174308831203133D027E
:1007D000031DEF2BC01DEF2B83120317481083124C
:1007E00003174818062C4814C81043088312031333
:1007F000C50083120317440883120313C400DB01EE
:100800003708EF003608F000CD144D140130080011
:10081000831203174810C22A83222C3C031D0C2C80
:10082000080083222A3C031D112C83228322832269
:10083000832208005503590784000008D7005A088E
:10084000840757088000D50B1A2C0800C8261F27DC
:1008500083120313203084000030D500302CD50AD9
:100860005508273C031C382C00085C27840A2F2CD1
:100870006F2C0A305C270D305C27831203132C3059
:10088000D700432CD70A5708393C031C4E2C570875
:10089000831203178D0050276027422C5C276F2C92
:1008A000831203132C30D700562CD70A5708393C33
:1008B000031C632C5708831203178D008312031344
:1008C00074275C27552C6F2CBC266F2C83120313C6
:1008D0004F305C274B305C276F2CB0266F2C831277
:1008E00003130A305C270D305C2783120313651C49
:1008F000772C7421752C051532268B26CF2883166C
:1009000003178230A000A030A1008430A2009830EC
:10091000A3006230A4006030A500E030A60083127E
:1009200003132830D9007F30DA000730D500550393
:100930005907840083130008D7005A0884078317D7
:10094000570880000310800DD50B972C8313DF26EA
:10095000831603172E08B03C031DB22C2D148316EA
:100960000317E916831603170330BC00F030BD00EF
:100970002F3083120313401ECF2C83160317C7009A
:10098000831203132F0883160317D1002130BE00F2
:100990002F30D2004130D4003D30D500D52C831605
:1009A00003172F30C9003A30BE0083160313831299
:1009B0000313C01FE12C401EDF2C3230E02C3530F9
:1009C000E22C3B3083160313AE002530A400A601B1
:1009D000A60AA70183120313340883160313A80081
:1009E0006E25A80BF02C72257225FF30A900AA00F5
:1009F0008317A030840083160317E91E082D831681
:100A000003130E30A8004525BC3084001C30AE0214
:100A1000831603132E08A800452583120313C01F55
:100A2000362D831203173D084B25831203173E080A
:100A30004B25831203173F084B252F304B2583127C
:100A4000031740084B258312031741084B258312D7
:100A5000031742084B2583120313401E312D093022
:100A6000322D063083160313A80045258313831601
:100A700003132909AF002A094B252F084B25033002
:100A8000A8007225A80B412D080000084B25840AF8
:100A9000A80B452D080083160313AB005F25083013
:100AA000AC0001302B05AD007E252708053A031D5B
:100AB0005B2DAD017E25AB0CAC0B512D0800AA06B9
:100AC0000830AC000310A90CAA0C031C6B2D843059
:100AD000A9060830AA06AC0B622D08008316031382
:100AE0007E30732D7E30AB000830AC0001302B051A
:100AF000AD007E25AB0CAC0B762D0800A70A2D1897
:100B0000842D0130A606A701261C8B2D1430A300CE
:100B10001030A5008F2D8B30A3001D30A50083164B
:100B2000A1012108031D952D912DA1030800A225E7
:100B3000A225A225A225A225A225A225A225A2257D
:100B4000A225080083120313D730CF00FF30CA005C
:100B5000A92DAA2DAB2DCA0BA82DAE2DAF2DCF0BD5
:100B6000A62DFF30CA000000CA0BB32DB72D080018
:100B7000061006148511080083120313C80006141A
:100B800085110511491B8515B825C91A8515B82584
:100B9000491A8515B825C9198515B8254919851526
:100BA000B825C9188515B82549188515B82585159E
:100BB0000610061405158511C81B8515B825481B98
:100BC0008515B825C81A8515B825481A8515B8257C
:100BD000C8198515B82548198515B825C81885156B
:100BE000B82548188515B82500348312031313302F
:100BF000C9000030BC25B1251330C9000130BC2527
:100C00000030C9001B30BC25B125B125B125B12567
:100C10000030C9001930BC25B125B1250030C9000C
:100C20001130BC25B1250030C9000130BC250B3086
:100C3000C9003308BC25831203130510B125003405
:100C4000831203130514831203130B30C900003001
:100C5000BC250030C9001B30BC250030C9000F3056
:100C6000BC2500340030C9001A30BC250030C90052
:100C70001B30BC25A2250130C9003008BC2502303C
:100C8000C9003108BC250330C9003208BC25043036
:100C9000C9003008BC250530C9003108BC25063024
:100CA000C9003208BC250730C9000030BC25083017
:100CB000C9003230BC25691E622E0930C900F330EC
:100CC000BC25662E0930C9008130BC250A30C90018
:100CD0000030BC250B30C9000030BC250C30C900E9
:100CE0004830BC250D30C9001030BC250E30C9007D
:100CF0002630BC251130C9001B30BC251330C9007B
:100D00000130BC251C30C9004030BC254230C90030
:100D10002530BC250034831203130E30C900663021
:100D2000BC25F525691E992E0930C900F330BC2574
:100D30009D2E0930C9008130BC250B30C900003020
:100D4000BC250E30C900E630BC25A2250E30C900F6
:100D50006630BC25A2250B30C9003308BC25003401
:100D6000D5015508BC20FF390319BB2E5C2783121F
:100D70000313D50AB12E0800D5015508B620FF3956
:100D80000319C72E5C2783120313D50ABD2E080052
:100D900083120313203084000030D700D02ED70AEE
:100DA0005708223C031CDE2E5708831203178D00C0
:100DB0008312031374278000840ACF2E0800831245
:100DC0000313AE30840083172C30D700E82ED70AE7
:100DD0005708393C031CF42E5708831203178D0063
:100DE00074278000840AE72E0800203084008030B9
:100DF000D700FB2ED70A57088E3C031C092F570833
:100E0000831203178D008312031300086027840ADE
:100E1000FA2E0800203084000030D700102FD70AA7
:100E20005708223C031C1E2F5708831203178D00FE
:100E30008312031300086027840A0F2F080083160B
:100E4000031310309B0083120313A1309F008316FD
:100E50000313C0309F00B125831203131F151F1900
:100E60002F2F831203131E08C600831603131E08B8
:100E700083120313C70090309F00831603139B0156
:100E80009F01831203139F010800D901D501D515D5
:100E9000DA0C0318D907D90CDA0CD50B492F080046
:100EA0008A153A268A1108008A153E268A110800FA
:100EB0008A1516268A1108008A1557268A110800F5
:100EC000831203178C008B13831603178C130C15D6
:100ED00055308D00AA308D008C148C186D2F0C1598
:100EE0008B17831203130800831603178C130C143B
:0C0EF000831203170C0883120313080080
:1010000082072434473450344734473441342C3435
:101010003034333433343634393431342E3430349C
:1010200030342C3433343434313432342E34333499
:101030003434353436342C344E342C343134323468
:101040003334343435342E34363437343834393458
:101050002C3457342C3431342C34303434342C3454
:1010600032342E34363439342C3430343034313454
:10107000303430342C344D342A3431343234333437
:10108000343400348316031783120608ED398600C2
:101090008316900194019301003091000130A0006B
:1010A0005228A00A2008803C031C682801309800C0
:1010B0005A28980A1808403C031C63288316031713
:1010C0000030042359282E30572683160317512841
:1010D00083160317EF1C8B28831603170130A0001B
:1010E0007228A00A2008803C031C88280130980040
:1010F0007A28980A1808403C031C83288316031793
:1011000000300423792825305726831603177128C9
:101110008316031736238A116F2C83160317EF1CCF
:10112000932831309428303057268A116F2C83123F
:1011300003130608ED39860083160317003090006C
:101140001F309400FD3093006B219D003F309400D0
:10115000A5309100562119300822831603171F303D
:1011600094005A309100562119300822831203133B
:101170000608ED3986008316031790013F3094006E
:10118000FD3093006B219C00EF011F3094001D087F
:10119000910056211C08A53C031DD728EF143130BF
:1011A0005726F830831603179C003F30DE28303076
:1011B0005726F830831603179C001F308316031739
:1011C0009D00940193018A117828831603178312D6
:1011D0000608ED39860083160317003090003A2682
:1011E0008316031794003A268316031793003A26B2
:1011F0008316031791005621193008228A116F2C8B
:101200008316031783120608ED3986008316031729
:1012100000309000831203133A26831603179400BC
:101220003A26831603179300A03084008317862183
:10123000A03084000008840A8A1557260008840A12
:101240008A1557260008840A8A1557260008840A3A
:101250008A1557260008840A8A1557260008840A2A
:101260008A1557260008840A8A1557260008840A1A
:101270008A15572683138A116F2C8316031783123E
:101280000608ED398600831603170030900083129C
:1012900003133A268316031794003A26831603177E
:1012A00093006B218A1557268A116F2CE6210310B3
:1012B000100DA0389600CA21DE2114089600CA211C
:1012C000DE2113089600CA21DE2111089600CA21EA
:1012D000DE21F1210800E6210310100DA038960050
:1012E000CA21DE2114089600CA21DE2113089600C7
:1012F000CA21DE21E6210310100DA1389600CA2173
:10130000DE21B121DE21F12117080800E6210310BA
:10131000100DA0389600CA21DE2114089600CA21BB
:10132000DE2113089600CA21DE21E6210310100DEC
:10133000A1389600CA21DE2101309900A029990A1E
:101340001908073C031CAA29B121E22117088000D3
:10135000840A9F29B121DE21F12117088000840A27
:101360000800970108309500861401220616012214
:101370008312861CBC29C02983160310970DC5292A
:1013800083160310970D970AC52906120122950BA3
:10139000B6290800083095000310960D031CD129CA
:1013A000D72986100122FC2186140122DB2986140C
:1013B0000122FC21DB29950BCC290800861401228F
:1013C000FC21080086100122FC21080006120122DF
:1013D000861401220616012286100122061201221D
:1013E0000800061201228610012206160122861428
:1013F000012206120122080006160122061201220D
:10140000080006309A0000009A0B032A0800FA3000
:10141000831603179900FF309A0006309B009B0B40
:101420000F2A9A0B0D2A990B0B2A0800831203131B
:101430008317401A1D2ACA301E2AC830840083161A
:1014400003170008EB00840A0008EC00840A000877
:10145000ED00840AC822DC00E322DD00840AE322D6
:10146000DE0083120313401E382A6B30840083137E
:1014700083160317EE01E322DF0083175C080423C1
:101480005D0804235E0804235F08691D482A80382C
:10149000042383120313401A4F2ABF30502ABF304F
:1014A000840083160317E322DC00E322DD00840AB4
:1014B000E322DE0083120313401E612A6930840098
:1014C000831383160317E322DF0083175C080423CA
:1014D0005D0804235E0804235F08E91C702A803835
:1014E000042383120313401A772AD630782AD63081
:1014F0008400831603170008EB00840A30306B0267
:10150000DC00E322DD00E322DE005C0804235D084A
:1015100004235E080423831603133108831603177C
:101520000423831203174308831603170423362367
:1015300083160317EF1CB12A1308EF3C031DB02AD2
:1015400014083F3C031DB02A83120313401CAD2A2C
:101550008316031793019401B02A831603176F149F
:10156000C52A1308F13C031DC52A14081F3C031D9E
:10157000C52A83120313401CC22A83160317930142
:101580009401C52A831603176F1483138A11172930
:1015900030306B02031C0301EE000310EE0DEE0D64
:1015A000EE07EE0D30306C02031C0301EE076E08EF
:1015B000EE0DEE0DEE07EE0D30306D02031C030153
:1015C000EE076E0808000008EC00840A0008ED0031
:1015D000840AEE01D222080083160317831206083C
:1015E000ED3986008316E6210310100DA038960011
:1015F000CA21E22114089600CA21E22113089600AC
:10160000CA21E221EF17080096006F1C082B080082
:10161000831603171608EF1B112B9700EC221708EF
:10162000960083160317CA21E221831603171308B5
:101630003F393F3C031D1F2B831603173623E91F39
:101640002F2B13081C02031D2F2B14081D02031D32
:101650002F2B83160317EF1F2E2B36236F14930A9D
:101660001308003C031D352B940A08006F1C392B0E
:101670000800F121EF13831603171930082283168F
:101680000317080083160317E91B052C83120313A5
:101690008317401A4D2BD6304E2BD630840083163C
:1016A0000317E101E20130300002E107E10DE10D35
:1016B000E107E10D840A30300002E1070724840AC3
:1016C00030300002E401E3006308E1076408031816
:1016D000640AE2070724840A30300002E401E300D0
:1016E0006308E10764080318640AE2070724840A10
:1016F00030300002E401E3006308E10764080318E6
:10170000640AE20783160317691BA02B83160313D1
:101710003108033C03189C2B83160317EA0A6A0856
:10172000023C031D9B2BEA0169178316031761080E
:10173000E5006208E6009F2B83160317EA01052CDB
:10174000831603133108033C0318052C8316031773
:101750006430E3000030E4006508E307660803181E
:10176000660AE4076308E7006408E8006108E70226
:101770006208031C620AE80267086804031DC22BA2
:10178000EA0ACA2B0318C82BEA0A76305726CA2B56
:10179000EA016917831603176A083F39033C031DE2
:1017A000052CEA016913E91713089C0014089D0031
:1017B0000430E3000130E40063089C026408031C69
:1017C000640A9D029D1FEA2BEF1CE82B1130E92BC8
:1017D0000F309C021D08EF1CEF2B3F39F02B1F39F7
:1017E0009D001308EB001408EC00FE3093001F303E
:1017F000EF1CFB2B3F3094001D0804231C0804231E
:1018000036236B0893006C0894008A11092961083B
:10181000E3006208E4000310E10DE20D0310E10DA6
:10182000E20D6308E10764080318640AE207031085
:06183000E10DE20D0800CD
:101C0000572683120313080083120313E301E5012F
:101C10008316031301178B178B1583120313080008
:101C20000B120800E600E60B132E080083120313C4
:101C30006510E514E401FF3012260830E700861F26
:101C40000310861B0314A9301226E40CE70B1F2E89
:101C5000861F2E2E6408E3006514E5100800831229
:101C60000313861B312E342E352E362E372E382E6A
:101C7000392E162E83120313651C3C2E8312031378
:101C800063086510080083120313E4008B1303102C
:101C90000930E700031C061303180617A9301226A3
:101CA000E40CE70B4A2E0617AC301226080083120C
:101CB0000313E4008B1303100930E700031C061321
:101CC00003180617A9301226E40CE70B5E2E061740
:081CD000AC3012268B1708004E
:101D000083120313DB0A5B08583C031D942EDB018E
:101D1000C50A45083C3C031D942EC501C40A44086D
:101D2000003C031D942EC30A08008316A001A101E4
:101D300021305726831203130030D700A02ED70A74
:101D40005708053C031CB42EB726831203136518ED
:101D5000AA2EB32E3E2683120313423A031DB22E3F
:101D6000002FB32E423A9F2E583057260800831278
:101D70000313D730CF00FF30CA00BE2EBF2EC02EB7
:101D8000CA0BBD2EC32EC42ECF0BBB2EFF30CA00F4
:0A1D90000000CA0BC82ECC2E08007C
:101E00008312031300309000920004268B13831278
:101E10000313E8014B3043262F26523A031D142F9B
:101E20003F2737275927362F523A583A031D212F7B
:101E30003F277E2737270310831203178F00B5270C
:101E4000362F583A573A031D2C2F3F277E27372726
:101E50004F278E279627362F573A453A031D352FA1
:101E60003F2737274F278E27362F453A072F2F2614
:101E7000680203193E2F43304326002F08002F2607
:101E8000E039831203178D0083120313E8072F260E
:101E9000831203178F0083120313E80708008312CD
:101EA00003170F080E3C031C562F08005230432620
:101EB000002F83120313E801831603172030E0007C
:101EC000831603178C170C140000000083120317ED
:101ED0000C0883120313E8074326831203170E0826
:101EE00083120313E8074326831203178D0A831610
:101EF0000317E00B602F680843260800A030840019
:101F00008317831603174030E0002F26E807800070
:101F1000840A83160317E00B852F08008316031726
:101F20008C170C16E127831203130800831603177E
:101F30008C170C12A03084008317831603172030EF
:101F4000E0008312031700088C00840A00088E004A
:101F5000840AE127831203178D0A83160317E00B07
:101F6000A12F8313831203130800831603178C1306
:101F7000A03084008317831603172030E0008312FB
:101F8000031700088C00840A840AD12783120317E0
:101F90008D0A83160317E00BBF2F831383120313DD
:101FA00008008B13831603170C1555308D00AA30CB
:101FB0008D008C148C18DA2F0C158B1783120313D9
:101FC0000800831603170C158B1355308D00AA30AB
:0C1FD0008D008C14000000000C110800B3
:02400E00023F6F
:02401000FC3F73
:10420000F400F400010084008400010000000000BC
:104210004B00370052004B005400200001002D00DD
:10422000420014002500FF000A0003000100020004
:104230000000A60000006400000000006400000010
:10424000310002004400000000000000FE00FE00FB
:104250005A005A005A005A00B000920088008A00A2
:10426000620040006200AE00920088008A00640094
:0442700040006300A7
:1043000000000000010023004B0037005800590056
:0E4310005A00200031000000230000002300AE
:00000001FF
